:10000000031E080086015F308C000D3084008001E3
:10001000840A8C0B07282C282120840007398406A9
:100020000310840C840C840C041A841704128A01B3
:10003000820701340234043408341034203440344C
:10004000803407398A018207303431343234333412
:1000500034343534363437340330392301309200A8
:1000600006303523BB223030E823D0230030B123C3
:10007000031D25290C08D0235730B123031D472821
:100080000C08D0231530B123031DAB2830280630CF
:1000900039230130F0230230A8005830EA2203301F
:1000A000352301309100BB226B200130F023023058
:1000B000A8000F08EA221108D0239B2322089100F0
:1000C0000130C023031D68288B30A7230319532850
:1000D00003303923302801308D008F01023039235D
:1000E00001308E000C08D0230D08802322089000D8
:1000F0001008D0230D08B123031D812804303523B7
:10010000832804303923023035233530E823D023C7
:100110000130B123031D8D2893280F08D0230D082B
:100120008B2322088F00023039230D08D0230230A0
:100130006D2322088D000E08D0239B2322088E00F9
:100140000130C023031DA8280830A72303197228F3
:1001500004303923F52B0630392301304023013098
:10016000F0230230A8001330EA2201308E00BB22B7
:100170000E08D0239B2322088E000130C023031DCC
:10018000C5283230A7230319B72801304023C222E3
:100190000030F0230230A800CC228C00CC228C004E
:1001A000CC228C00CC228C00CC228C00CC22920061
:1001B000CC22930001308E00BB220E08D0239B235B
:1001C00022088E000130C023031DEA280730A72330
:1001D0000319DC280030F0230230A800CC228C0068
:1001E000CC228E0001304023C222130898008422C2
:1001F0000C08D0230130B123031D05290C08D0239E
:100200000230B123031D182930281208D0230A30E8
:100210006D23220892001D08D0230A30562322089D
:100220009D001208D0231D088B232208920030283D
:100230001208D02364306D23220892001208D023C4
:100240001D088B232208920030283030E823D02369
:100250000030B123031D25290630392364304023A3
:100260001208D0230030B123031D3B291208D023EC
:10027000C830A723031D3D293F29013092001208F1
:10028000D02310305623220893001308D0231030B7
:100290006D23220894001208D02314088723220813
:1002A00094001408D02308306D2322089400140809
:1002B000D02304308B23220894000330352391018E
:1002C00001308A001108FA3E03187329063E6A219C
:1002D0008C00732982078134523400340034003496
:1002E0007129130808006B201108D0239B232208D2
:1002F00091000030C023031D81290530A723031975
:1003000060298C01013091006B201108D0239B23C0
:10031000220891000130C023031D92291408A7234D
:10032000031984296B200F0895006B200F08960095
:100330006B200F0897006B200F0898006B200F08A8
:10034000D02301308B2322089E0003303923013053
:10035000F0230230A8001630EA22BB220C08D0237A
:100360001330B623031D3028013040231508D02355
:100370000130A50000306E234430DA234430D3230B
:1003800016088B234430DA234508CD004408CC00FE
:100390001708D0230130A50000306E234630DA2341
:1003A0004630D32318088B234630DA231E08D02387
:1003B0003330AC23031DEF294630D323013087238C
:1003C0004E30DA233230D0231E08872322089F00C4
:1003D0008030D0231F08872322089F00F92947086F
:1003E000CF004608CE001E08D023323087232208D3
:1003F0009F00033035239901910102308A001108D2
:10040000F93E0318132A073E07228C00132A82079D
:1004100081345234003400340F2A112A0034150874
:100420000800160808006B201108D0230A30AC23FE
:10043000031D1B2A502A0130F0230230A8000F08A8
:10044000EA221908D02301308B2322089900443076
:10045000D3234E30E123B3230319342A1908D023C0
:100460001F08B123031D422A1908D0233230B123BB
:100470000319412A4430D3234C30E123B323031D15
:10048000422A502ABB22013040230C08D0232130BD
:10049000B123031D4C2A502AC222BB220130402323
:1004A0001108D0239B23220891000030C023031D94
:1004B0005D2A8930A7230319FD29033039234430ED
:1004C000D32301308B234430DA234430D323463006
:1004D000E123A923031D30284430D3230130A50094
:1004E00000305723220895001508D0230130A500BD
:1004F00000306E234830DA234430D3234830E123E0
:10050000892322089600F9299C0190309A001A0844
:10051000D02309308B2322089B001808D0231A0807
:10052000AC230319992A1808D0231B08BB23031DE9
:100530009A2AA02A1808D0231C088B2322089D0081
:100540001C08D02306308B2322089C001A08D023D5
:100550001030872322089A009030A723031DB42A65
:100560000030C0230319872A1D08D0233630872383
:1005700022089D00F52B0030F0230230A800CC2289
:100580008C00F52B0130F0230230A8000630EA225F
:10059000F52B07304E23C92A270884008417260824
:1005A00080046400E0220318D12A13230830AA0033
:1005B0001523E022AB0CAA0BD82A15232B08080020
:1005C0002708840026080005281926060310031DA5
:1005D000031408006400AB000930AA000310F522E0
:1005E000AB0CAA0BEF2A0314F52A2708840026086F
:1005F000A81D072B281D0301000626058006841769
:100600002608031C0301000626058006172B0000A0
:10061000031C0301281926060006260580068417F8
:1006200026098005172B28171C2B0330182B0230A6
:10063000FF3E031D182B281303308A00280D0639AE
:1006400082070830292B1030292B0230292B40300B
:10065000292BA900281BA90C322B0C30FF3E031DAF
:100660002E2B0000A90B2D2B08000C20FF3A800533
:100670003D2B0C2080043C2BFF3A84178005F52B82
:10068000A301A2009923640023082204031908008F
:10069000F730FF3E031D492B9B23432B831607395D
:1006A000F83881006300FF308100F52BA501A4001C
:1006B0001030AB00AA01A9010314A20DA30DA90DCE
:1006C000AA0D9F2329308E23031C22109F2329303B
:1006D000221C8E23AB0B5C2BF52BA501A40029302B
:1006E000DA23A301A2012A0829040319F52B031018
:1006F000AA0CA90C03188D230310A40DA50D732BB0
:10070000A501A4002408A2052508A305F52BA50131
:10071000A4009F238D2BA501A4002230840024086F
:1007200080072508840F00000318013E031C800782
:10073000F52BA309A209A20A0319A30A0800A423FE
:10074000A40A0319A50AF52BA509A409F52BA501EF
:10075000A400C5230139F52BA501A400C523033945
:10076000F52BA501A400C5230239F52BA501A40092
:10077000C5230539F52BA501A400C5230639F52BA2
:10078000A501A400C5230439F52B25082302031D68
:10079000CD2B2408220203190234031C0434013433
:1007A000A301A200F52B84000008A200840A00081F
:1007B000A300F52B840022088000840A230880000F
:1007C000F52B84000008A400840A0008A500F52B7E
:1007D0000D20A9000005841B2906031900340134EB
:1007E00021200D20A6000408A70083126400080041
:1007F000FF3FFF3FFF3FFF3FFF3FFF3FFF3FFF3F09
:084000000F000F000F000F007C
:02400E000D00A3
:10420000FF00FF00FF00FF00FF00FF00FF00FF00B6
:10421000FF00FF00FF00FF00FF00FF00FF00FF00A6
:10422000FF00FF00FF00FF00FF00FF00FF00FF0096
:10423000FF00FF00FF00FF00FF00FF00FF00FF0086
:10424000FF00FF00FF00FF00FF00FF00FF00FF0076
:10425000FF00FF00FF00FF00FF00FF00FF00FF0066
:10426000FF00FF00FF00FF00FF00FF00FF00FF0056
:10427000FF00FF00FF00FF00FF00FF00FF00FF0046
:00000001FF
